BL51 BANKED LINKER/LOCATER V5.03                                                        06/21/2006  12:48:46  PAGE 1


BL51 BANKED LINKER/LOCATER V5.03, INVOKED BY:
C:\KEIL\C51\BIN\BL51.EXE STARTUP.obj, pcf8563_demo1.obj, iic.obj, pcf8563.obj, delay.obj TO pcf8563_demo1 RAMSIZE (256) 
>> CODE (0X0000-0X1FFF)


MEMORY MODEL: SMALL


INPUT MODULES INCLUDED:
  STARTUP.obj (?C_STARTUP)
  pcf8563_demo1.obj (PCF8563_DEMO1)
  iic.obj (IIC)
  pcf8563.obj (PCF8563)
  delay.obj (DELAY)
  C:\KEIL\C51\LIB\C51S.LIB (?C?CLDPTR)
  C:\KEIL\C51\LIB\C51S.LIB (?C?CSTPTR)
  C:\KEIL\C51\LIB\C51S.LIB (PRINTF)
  C:\KEIL\C51\LIB\C51S.LIB (?C?CLDOPTR)
  C:\KEIL\C51\LIB\C51S.LIB (?C?PLDIIDATA)
  C:\KEIL\C51\LIB\C51S.LIB (?C?CCASE)
  C:\KEIL\C51\LIB\C51S.LIB (PUTCHAR)


LINK MAP OF MODULE:  pcf8563_demo1 (?C_STARTUP)


            TYPE    BASE      LENGTH    RELOCATION   SEGMENT NAME
            -----------------------------------------------------

            * * * * * * *   D A T A   M E M O R Y   * * * * * * *
            REG     0000H     0008H     ABSOLUTE     "REG BANK 0"
                    0008H     0018H                  *** GAP ***
            BIT     0020H.0   0001H.1   UNIT         _BIT_GROUP_
                    0021H.1   0000H.7                *** GAP ***
            DATA    0022H     001EH     UNIT         _DATA_GROUP_
            IDATA   0040H     0001H     UNIT         ?STACK

            * * * * * * *   C O D E   M E M O R Y   * * * * * * *
            CODE    0000H     0003H     ABSOLUTE     
                    0003H     07FDH                  *** GAP ***
            CODE    0800H     035CH     UNIT         ?PR?PRINTF?PRINTF
            CODE    0B5CH     008EH     UNIT         ?C?LIB_CODE
            CODE    0BEAH     0081H     INBLOCK      ?PR?MAIN?PCF8563_DEMO1
            CODE    0C6BH     0060H     INBLOCK      ?PR?_I2C_SEQRD?IIC
            CODE    0CCBH     0057H     INBLOCK      ?PR?_RTCGETDATE?PCF8563
            CODE    0D22H     0055H     INBLOCK      ?PR?_RTCGETTIME?PCF8563
            CODE    0D77H     0047H     UNIT         ?CO?PCF8563_DEMO1
            CODE    0DBEH     0046H     INBLOCK      ?PR?_I2C_SENDBYTE?IIC
            CODE    0E04H     0043H     INBLOCK      ?PR?_I2C_SEQWR?IIC
            CODE    0E47H     0027H     UNIT         ?PR?PUTCHAR?PUTCHAR
            CODE    0E6EH     0023H     INBLOCK      ?PR?I2C_RCVBYTE?IIC
            CODE    0E91H     0020H     INBLOCK      ?PR?_DELAYMS?DELAY
            CODE    0EB1H     001DH     INBLOCK      ?PR?_RTCSETDATE?PCF8563
            CODE    0ECEH     001AH     INBLOCK      ?PR?_RTCSETTIME?PCF8563
            CODE    0EE8H     0018H     INBLOCK      ?PR?I2C_ACK?IIC
            CODE    0F00H     0017H     INBLOCK      ?PR?RTCINIT?PCF8563
            CODE    0F17H     0013H     INBLOCK      ?PR?I2C_START?IIC
            CODE    0F2AH     0012H     INBLOCK      ?PR?_DELAYUS?DELAY
BL51 BANKED LINKER/LOCATER V5.03                                                      06/21/2006  12:48:46  PAGE 2


            CODE    0F3CH     0011H     INBLOCK      ?PR?I2C_STOP?IIC
            CODE    0F4DH     000FH     INBLOCK      ?PR?_RTCBCD2DEC?PCF8563
            CODE    0F5CH     000DH     INBLOCK      ?PR?INIT_UART?PCF8563_DEMO1
            CODE    0F69H     000CH     UNIT         ?C_C51STARTUP



OVERLAY MAP OF MODULE:   pcf8563_demo1 (?C_STARTUP)


SEGMENT                                BIT_GROUP          DATA_GROUP 
  +--> CALLED SEGMENT               START    LENGTH     START    LENGTH
-----------------------------------------------------------------------
?C_C51STARTUP                       -----    -----      -----    -----
  +--> ?PR?MAIN?PCF8563_DEMO1

?PR?MAIN?PCF8563_DEMO1              -----    -----      0022H    0007H
  +--> ?PR?INIT_UART?PCF8563_DEMO1
  +--> ?PR?RTCINIT?PCF8563
  +--> ?PR?_RTCSETTIME?PCF8563
  +--> ?PR?_RTCSETDATE?PCF8563
  +--> ?PR?_RTCGETTIME?PCF8563
  +--> ?CO?PCF8563_DEMO1
  +--> ?PR?PRINTF?PRINTF
  +--> ?PR?_RTCGETDATE?PCF8563
  +--> ?PR?_DELAYMS?DELAY

?PR?RTCINIT?PCF8563                 -----    -----      0029H    0002H
  +--> ?PR?_I2C_SEQWR?IIC

?PR?_I2C_SEQWR?IIC                  -----    -----      0031H    0007H
  +--> ?PR?I2C_START?IIC
  +--> ?PR?_I2C_SENDBYTE?IIC
  +--> ?PR?I2C_STOP?IIC

?PR?_RTCSETTIME?PCF8563             -----    -----      0029H    0003H
  +--> ?PR?_I2C_SEQWR?IIC

?PR?_RTCSETDATE?PCF8563             -----    -----      0029H    0008H
  +--> ?PR?_I2C_SEQWR?IIC

?PR?_RTCGETTIME?PCF8563             -----    -----      0029H    000CH
  +--> ?PR?_I2C_SEQRD?IIC
  +--> ?PR?_RTCBCD2DEC?PCF8563

?PR?_I2C_SEQRD?IIC                  -----    -----      0039H    0007H
  +--> ?PR?I2C_START?IIC
  +--> ?PR?_I2C_SENDBYTE?IIC
  +--> ?PR?I2C_RCVBYTE?IIC
  +--> ?PR?I2C_ACK?IIC
  +--> ?PR?I2C_STOP?IIC

?PR?I2C_ACK?IIC                     0020H.0  0000H.1    -----    -----

?PR?PRINTF?PRINTF                   0020H.0  0001H.1    0029H    0014H
  +--> ?PR?PUTCHAR?PUTCHAR

BL51 BANKED LINKER/LOCATER V5.03                                                      06/21/2006  12:48:46  PAGE 3


?PR?_RTCGETDATE?PCF8563             -----    -----      0029H    0010H
  +--> ?PR?_I2C_SEQRD?IIC
  +--> ?PR?_RTCBCD2DEC?PCF8563



SYMBOL TABLE OF MODULE:  pcf8563_demo1 (?C_STARTUP)

  VALUE           TYPE          NAME
  ----------------------------------

  -------         MODULE        ?C_STARTUP
  C:0F69H         SEGMENT       ?C_C51STARTUP
  I:0040H         SEGMENT       ?STACK
  C:0000H         PUBLIC        ?C_STARTUP
  D:00E0H         SYMBOL        ACC
  D:00F0H         SYMBOL        B
  D:0083H         SYMBOL        DPH
  D:0082H         SYMBOL        DPL
  N:0000H         SYMBOL        IBPSTACK
  N:0100H         SYMBOL        IBPSTACKTOP
  N:0080H         SYMBOL        IDATALEN
  C:0F6CH         SYMBOL        IDATALOOP
  N:0000H         SYMBOL        PBPSTACK
  N:0000H         SYMBOL        PBPSTACKTOP
  N:0000H         SYMBOL        PDATALEN
  N:0000H         SYMBOL        PDATASTART
  N:0000H         SYMBOL        PPAGE
  N:0000H         SYMBOL        PPAGEENABLE
  D:00A0H         SYMBOL        PPAGE_SFR
  D:0081H         SYMBOL        SP
  C:0F69H         SYMBOL        STARTUP1
  N:0000H         SYMBOL        XBPSTACK
  N:0000H         SYMBOL        XBPSTACKTOP
  N:0000H         SYMBOL        XDATALEN
  N:0000H         SYMBOL        XDATASTART
  C:0000H         LINE#         92
  C:0F69H         LINE#         99
  C:0F6BH         LINE#         100
  C:0F6CH         LINE#         101
  C:0F6DH         LINE#         102
  C:0F6FH         LINE#         151
  C:0F72H         LINE#         155
  -------         ENDMOD        ?C_STARTUP

  -------         MODULE        PCF8563_DEMO1
  C:0000H         SYMBOL        _ICE_DUMMY_
  C:0BEAH         PUBLIC        main
  D:0098H         PUBLIC        SCON
  D:0089H         PUBLIC        TMOD
  D:0088H         PUBLIC        TCON
  D:008DH         PUBLIC        TH1
  C:0F5CH         PUBLIC        init_uart
  -------         PROC          INIT_UART
  C:0F5CH         LINE#         30
  C:0F5CH         LINE#         31
  C:0F5CH         LINE#         32
BL51 BANKED LINKER/LOCATER V5.03                                                      06/21/2006  12:48:46  PAGE 4


  C:0F5FH         LINE#         33
  C:0F62H         LINE#         34
  C:0F65H         LINE#         35
  C:0F68H         LINE#         36
  -------         ENDPROC       INIT_UART
  -------         PROC          MAIN
  -------         DO            
  D:0022H         SYMBOL        hour
  D:0023H         SYMBOL        min
  D:0024H         SYMBOL        sec
  D:0025H         SYMBOL        date
  D:0026H         SYMBOL        dow
  D:0027H         SYMBOL        month
  D:0028H         SYMBOL        year
  -------         ENDDO         
  C:0BEAH         LINE#         43
  C:0BEAH         LINE#         44
  C:0BEAH         LINE#         47
  C:0BECH         LINE#         48
  C:0BEEH         LINE#         49
  C:0BF6H         LINE#         50
  C:0C01H         LINE#         52
  C:0C01H         LINE#         53
  C:0C01H         LINE#         54
  C:0C1BH         LINE#         55
  C:0C2CH         LINE#         56
  C:0C4FH         LINE#         57
  C:0C63H         LINE#         58
  C:0C69H         LINE#         59
  -------         ENDPROC       MAIN
  -------         ENDMOD        PCF8563_DEMO1

  -------         MODULE        IIC
  C:0000H         SYMBOL        _ICE_DUMMY_
  D:0090H         PUBLIC        P1
  C:0F3CH         PUBLIC        i2c_Stop
  C:0C6BH         PUBLIC        _i2c_SeqRd
  C:0E6EH         PUBLIC        i2c_RcvByte
  C:0E04H         PUBLIC        _i2c_SeqWr
  B:0090H.3       PUBLIC        SDA
  C:0DBEH         PUBLIC        _i2c_SendByte
  B:0090H.2       PUBLIC        SCL
  C:0EE8H         PUBLIC        i2c_Ack
  C:0F17H         PUBLIC        i2c_Start
  -------         PROC          I2C_START
  C:0F17H         LINE#         38
  C:0F17H         LINE#         39
  C:0F17H         LINE#         40
  C:0F19H         LINE#         41
  C:0F1BH         LINE#         42
  C:0F20H         LINE#         43
  C:0F22H         LINE#         44
  C:0F27H         LINE#         45
  C:0F29H         LINE#         46
  -------         ENDPROC       I2C_START
  -------         PROC          I2C_STOP
  C:0F3CH         LINE#         58
BL51 BANKED LINKER/LOCATER V5.03                                                      06/21/2006  12:48:46  PAGE 5


  C:0F3CH         LINE#         59
  C:0F3CH         LINE#         60
  C:0F3EH         LINE#         61
  C:0F40H         LINE#         62
  C:0F45H         LINE#         63
  C:0F47H         LINE#         64
  C:0F4CH         LINE#         65
  -------         ENDPROC       I2C_STOP
  -------         PROC          I2C_ACK
  B:0020H.0       SYMBOL        reply
  C:0EE8H         LINE#         80
  C:0EE8H         LINE#         81
  C:0EE8H         LINE#         82
  C:0EF1H         LINE#         83
  C:0EF4H         LINE#         84
  C:0EF6H         LINE#         85
  C:0EFBH         LINE#         86
  C:0EFDH         LINE#         87
  C:0EFFH         LINE#         88
  -------         ENDPROC       I2C_ACK
  -------         PROC          _I2C_SENDBYTE
  D:0007H         SYMBOL        c
  -------         DO            
  D:0006H         SYMBOL        i
  -------         ENDDO         
  C:0DBEH         LINE#         107
  C:0DBEH         LINE#         108
  C:0DBEH         LINE#         111
  C:0DC0H         LINE#         112
  C:0DC0H         LINE#         113
  C:0DD3H         LINE#         114
  C:0DD4H         LINE#         115
  C:0DD6H         LINE#         116
  C:0DDBH         LINE#         117
  C:0DDDH         LINE#         118
  C:0DE1H         LINE#         119
  C:0DE3H         LINE#         120
  C:0DE5H         LINE#         121
  C:0DE7H         LINE#         122
  C:0DF3H         LINE#         123
  C:0DFCH         LINE#         124
  C:0DFEH         LINE#         125
  C:0E00H         LINE#         126
  C:0E03H         LINE#         127
  -------         ENDPROC       _I2C_SENDBYTE
  -------         PROC          I2C_RCVBYTE
  -------         DO            
  D:0007H         SYMBOL        val
  D:0006H         SYMBOL        i
  -------         ENDDO         
  C:0E6EH         LINE#         139
  C:0E6EH         LINE#         140
  C:0E6EH         LINE#         141
  C:0E70H         LINE#         144
  C:0E72H         LINE#         146
  C:0E73H         LINE#         147
  C:0E73H         LINE#         148
BL51 BANKED LINKER/LOCATER V5.03                                                      06/21/2006  12:48:46  PAGE 6


  C:0E75H         LINE#         149
  C:0E7AH         LINE#         150
  C:0E7CH         LINE#         151
  C:0E7EH         LINE#         152
  C:0E82H         LINE#         153
  C:0E88H         LINE#         154
  C:0E8CH         LINE#         156
  C:0E8EH         LINE#         157
  C:0E90H         LINE#         158
  C:0E90H         LINE#         159
  -------         ENDPROC       I2C_RCVBYTE
  -------         PROC          _I2C_SEQWR
  D:0007H         SYMBOL        device
  D:0005H         SYMBOL        addrh
  D:0004H         SYMBOL        addrl
  D:0034H         SYMBOL        s
  D:0037H         SYMBOL        length
  -------         DO            
  D:0005H         SYMBOL        i
  -------         ENDDO         
  C:0E04H         LINE#         181
  C:0E06H         LINE#         182
  C:0E06H         LINE#         185
  C:0E08H         LINE#         186
  C:0E0DH         LINE#         187
  C:0E11H         LINE#         188
  C:0E11H         LINE#         189
  C:0E18H         LINE#         190
  C:0E18H         LINE#         191
  C:0E1FH         LINE#         192
  C:0E27H         LINE#         193
  C:0E27H         LINE#         194
  C:0E35H         LINE#         195
  C:0E40H         LINE#         196
  C:0E43H         LINE#         197
  C:0E45H         LINE#         198
  C:0E46H         LINE#         199
  -------         ENDPROC       _I2C_SEQWR
  -------         PROC          _I2C_SEQRD
  D:0004H         SYMBOL        device
  D:0005H         SYMBOL        addrh
  D:0003H         SYMBOL        addrl
  D:003CH         SYMBOL        s
  D:003FH         SYMBOL        length
  -------         DO            
  D:0005H         SYMBOL        i
  -------         ENDDO         
  C:0C6BH         LINE#         219
  C:0C6DH         LINE#         220
  C:0C6DH         LINE#         223
  C:0C6FH         LINE#         224
  C:0C74H         LINE#         225
  C:0C78H         LINE#         226
  C:0C78H         LINE#         227
  C:0C7FH         LINE#         228
  C:0C7FH         LINE#         229
  C:0C86H         LINE#         230
BL51 BANKED LINKER/LOCATER V5.03                                                      06/21/2006  12:48:46  PAGE 7


  C:0C88H         LINE#         232
  C:0C90H         LINE#         234
  C:0C9BH         LINE#         235
  C:0C9BH         LINE#         236
  C:0CA6H         LINE#         237
  C:0CAAH         LINE#         238
  C:0CB5H         LINE#         239
  C:0CB8H         LINE#         241
  C:0CC3H         LINE#         242
  C:0CC7H         LINE#         243
  C:0CC9H         LINE#         245
  C:0CCAH         LINE#         246
  -------         ENDPROC       _I2C_SEQRD
  -------         ENDMOD        IIC

  -------         MODULE        PCF8563
  C:0000H         SYMBOL        _ICE_DUMMY_
  D:0090H         PUBLIC        P1
  D:00B0H         PUBLIC        P3
  D:00A8H         PUBLIC        IE
  D:00B8H         PUBLIC        IP
  D:0098H         PUBLIC        SCON
  D:0088H         PUBLIC        TCON
  C:0CCBH         PUBLIC        _rtcGetDate
  C:0EB1H         PUBLIC        _rtcSetDate
  C:0D22H         PUBLIC        _rtcGetTime
  C:0F00H         PUBLIC        rtcInit
  D:00C8H         PUBLIC        T2CON
  C:0ECEH         PUBLIC        _rtcSetTime
  C:0F4DH         SYMBOL        _rtcBCD2DEC
  D:00D0H         PUBLIC        PSW
  -------         PROC          _RTCBCD2DEC
  D:0007H         SYMBOL        bcd
  -------         DO            
  D:0007H         SYMBOL        decimal_value
  -------         ENDDO         
  C:0F4DH         LINE#         65
  C:0F4DH         LINE#         66
  C:0F4DH         LINE#         69
  C:0F5BH         LINE#         71
  C:0F5BH         LINE#         72
  -------         ENDPROC       _RTCBCD2DEC
  -------         PROC          RTCINIT
  -------         DO            
  D:0029H         SYMBOL        s
  -------         ENDDO         
  C:0F00H         LINE#         88
  C:0F00H         LINE#         89
  C:0F00H         LINE#         92
  C:0F03H         LINE#         93
  C:0F05H         LINE#         94
  -------         ENDPROC       RTCINIT
  -------         PROC          _RTCSETTIME
  D:0007H         SYMBOL        sec
  D:0005H         SYMBOL        min
  D:0003H         SYMBOL        hour
  -------         DO            
BL51 BANKED LINKER/LOCATER V5.03                                                      06/21/2006  12:48:46  PAGE 8


  D:0029H         SYMBOL        s
  -------         ENDDO         
  C:0ECEH         LINE#         108
  C:0ECEH         LINE#         109
  C:0ECEH         LINE#         111
  C:0ED0H         LINE#         112
  C:0ED2H         LINE#         113
  C:0ED4H         LINE#         114
  -------         ENDPROC       _RTCSETTIME
  -------         PROC          _RTCSETDATE
  D:0007H         SYMBOL        day
  D:0005H         SYMBOL        dow
  D:0003H         SYMBOL        month
  D:002CH         SYMBOL        year
  -------         DO            
  D:002DH         SYMBOL        s
  -------         ENDDO         
  C:0EB1H         LINE#         128
  C:0EB1H         LINE#         129
  C:0EB1H         LINE#         131
  C:0EB3H         LINE#         132
  C:0EB5H         LINE#         133
  C:0EB7H         LINE#         134
  C:0EBAH         LINE#         135
  -------         ENDPROC       _RTCSETDATE
  -------         PROC          _RTCGETDATE
  D:0029H         SYMBOL        date
  D:002CH         SYMBOL        dow
  D:002FH         SYMBOL        month
  D:0032H         SYMBOL        year
  -------         DO            
  D:0035H         SYMBOL        s
  -------         ENDDO         
  C:0CCBH         LINE#         149
  C:0CD1H         LINE#         150
  C:0CD1H         LINE#         153
  C:0CE5H         LINE#         154
  C:0CF5H         LINE#         155
  C:0D05H         LINE#         156
  C:0D15H         LINE#         157
  -------         ENDPROC       _RTCGETDATE
  -------         PROC          _RTCGETTIME
  D:0029H         SYMBOL        sec
  D:002CH         SYMBOL        min
  D:002FH         SYMBOL        hour
  -------         DO            
  D:0032H         SYMBOL        s
  -------         ENDDO         
  C:0D22H         LINE#         171
  C:0D28H         LINE#         172
  C:0D28H         LINE#         175
  C:0D3CH         LINE#         176
  C:0D4CH         LINE#         177
  C:0D5CH         LINE#         178
  C:0D6CH         LINE#         180
  C:0D71H         LINE#         181
  C:0D74H         LINE#         183
BL51 BANKED LINKER/LOCATER V5.03                                                      06/21/2006  12:48:46  PAGE 9


  C:0D76H         LINE#         184
  -------         ENDPROC       _RTCGETTIME
  -------         ENDMOD        PCF8563

  -------         MODULE        DELAY
  C:0000H         SYMBOL        _ICE_DUMMY_
  D:0090H         PUBLIC        P1
  D:00B0H         PUBLIC        P3
  D:00A8H         PUBLIC        IE
  C:0E91H         PUBLIC        _DelayMs
  D:00B8H         PUBLIC        IP
  C:0F2AH         PUBLIC        _DelayUs
  D:0098H         PUBLIC        SCON
  D:0088H         PUBLIC        TCON
  D:00C8H         PUBLIC        T2CON
  D:00D0H         PUBLIC        PSW
  -------         PROC          _DELAYUS
  D:0006H         SYMBOL        N
  -------         DO            
  D:0004H         SYMBOL        x
  -------         ENDDO         
  C:0F2AH         LINE#         36
  C:0F2AH         LINE#         37
  C:0F2AH         LINE#         40
  C:0F3BH         LINE#         41
  -------         ENDPROC       _DELAYUS
  -------         PROC          _DELAYMS
  D:0006H         SYMBOL        msec
  -------         DO            
  D:0004H         SYMBOL        x
  D:0002H         SYMBOL        y
  -------         ENDDO         
  C:0E91H         LINE#         54
  C:0E91H         LINE#         55
  C:0E91H         LINE#         58
  C:0E9BH         LINE#         59
  C:0E9BH         LINE#         60
  C:0EA9H         LINE#         61
  C:0EB0H         LINE#         62
  -------         ENDPROC       _DELAYMS
  -------         ENDMOD        DELAY

  -------         MODULE        ?C?CLDPTR
  C:0B5CH         PUBLIC        ?C?CLDPTR
  -------         ENDMOD        ?C?CLDPTR

  -------         MODULE        ?C?CSTPTR
  C:0B75H         PUBLIC        ?C?CSTPTR
  -------         ENDMOD        ?C?CSTPTR

  -------         MODULE        PRINTF
  D:0029H         PUBLIC        ?_PRINTF517?BYTE
  D:0029H         PUBLIC        ?_PRINTF?BYTE
  D:0029H         PUBLIC        ?_SPRINTF517?BYTE
  D:0029H         PUBLIC        ?_SPRINTF?BYTE
  C:0862H         PUBLIC        _PRINTF
  C:0862H         PUBLIC        _PRINTF517
BL51 BANKED LINKER/LOCATER V5.03                                                      06/21/2006  12:48:46  PAGE 10


  C:085CH         PUBLIC        _SPRINTF
  C:085CH         PUBLIC        _SPRINTF517
  -------         ENDMOD        PRINTF

  -------         MODULE        ?C?CLDOPTR
  C:0B87H         PUBLIC        ?C?CLDOPTR
  -------         ENDMOD        ?C?CLDOPTR

  -------         MODULE        ?C?PLDIIDATA
  C:0BB4H         PUBLIC        ?C?PLDIIDATA
  -------         ENDMOD        ?C?PLDIIDATA

  -------         MODULE        ?C?CCASE
  C:0BC4H         PUBLIC        ?C?CCASE
  -------         ENDMOD        ?C?CCASE

  -------         MODULE        PUTCHAR
  C:0E47H         PUBLIC        _PUTCHAR
  -------         ENDMOD        PUTCHAR

*** WARNING L16: UNCALLED SEGMENT, IGNORED FOR OVERLAY PROCESS
    SEGMENT: ?PR?_DELAYUS?DELAY

******************************************************************************
* RESTRICTED VERSION WITH 0800H BYTE CODE SIZE LIMIT; USED: 0387H BYTE (44%) *
******************************************************************************

Program Size: data=40.1 xdata=0 code=1912
LINK/LOCATE RUN COMPLETE.  1 WARNING(S),  0 ERROR(S)
